:0600000088310028000019
:0800080083018A012000770842
:10001000A0007808A1007908A2007A08A3008B1E2E
:1000200013280B191C282008F7002108F8002208C3
:10003000F9002308FA00090080317F2902302100ED
:10004000C502031C3028203085007530840000086C
:10005000031930282E282C282D280000800B2B284F
:10006000200008002100C80148080F3C031CA728F5
:10007000C701C9014908073C031C9C28C601460862
:10008000C50020000D18522821004508133C031814
:100090004B2820005228C50A8530F700F70B4E2860
:1000A0004128200021004508143C031D6C28490804
:1000B000033C031869282730480784002030850056
:1000C0000318850A4708800001304807F800A9286E
:1000D0006C284808F800A92820000D1C7D28210064
:1000E00046089F3C0318762820007D28C60A8530E4
:1000F000F700F70B79286C28200021004608A03C67
:10010000031D8F28273048078400203085000318FE
:10011000850A4708800001304807F800A9284508EB
:10012000C5070310C70D4608450203189928471450
:100130009A284710C90A3A282730480784002030F7
:1001400085000318850A47088000C80A3428480833
:10015000F800200008002100C80148080F3C031CDB
:100160001629C701C9014908073C031C0B29C60110
:100170004608C50020000D18CB2821004508313C59
:100180000318C4282000CB28C50A8530F700F70BD8
:10019000C728BA28200021004508323C031DDD286D
:1001A000273048078400203085000318850A470857
:1001B000800001304807F800182920000D1CEE28A7
:1001C00021004608133C0318E7282000EE28C60A41
:1001D0008530F700F70BEA28DD28200021004608CB
:1001E000143C031D00292730480784002030850077
:1001F0000318850A4708800001304807F8001829CD
:100200000310C70D45080F3C031C08294710092996
:100210004714C90AB32827304807840020308500D6
:100220000318850A47088000C80AAD284808F80066
:100230002000080021000D1420000D1C2229003090
:10024000F8007D292100C20120000D183429210069
:100250004208773C03182E2920003429C20A643052
:10026000C50020001E20252921004208783C031DDE
:100270003E290030F80020007D292100C201200025
:100280000D1C502921004208773C03184929200001
:100290005029C20A8530F700F70B4C293F2920006E
:1002A00021004208783C031D5A290030F800200044
:1002B0007D2921004208143C0318662901302000E2
:1002C000D800322078082100C3006D2903302000B7
:1002D000D800AB2078082100C300C30803197B298C
:1002E00042083C3C031C7B294208133C031C7A292E
:1002F000C3177B2943174308F80020000800220099
:100300000D160D128B1220001A2178082100C00052
:10031000C0080319442A4008C20042083F39C500FA
:10032000C3014308013C031CCC290530430784006A
:10033000203085000318850A45080002031DCA29DC
:10034000C4014408C600450844020318C2292730E6
:1003500044078400203085000318850A0008C70080
:10036000430EF700F030F70577084407073E840096
:10037000203085000318850A00084702031DC229A2
:10038000C40AA32945084402031DCA2901304307B2
:10039000F800CE29C30A91290030F8007808BC0083
:1003A000BC080319442A3C08013A20000319DC293F
:1003B000033A03190D2A3E2AE208031DE6296108C3
:1003C000C73C031CE629E30A0319E40AE201E10140
:1003D000E408031DEF296308143C0318FD2958089D
:1003E000033C031DF82902302100C100FB29200035
:1003F00005302100C100002A200001302100C10089
:100400004108C103003A03190C2A200059087F3C17
:10041000031DD90A2100002A402AE208031D172AD9
:100420006108C73C031C172AE30A0319E40AE20126
:10043000E101E408031D202A6308143C03182E2A56
:100440005808033C031D292A04302100C1002C2A2E
:1004500020000A302100C100312A20000130210093
:10046000C1004108C103003A03193C2A2000D90801
:10047000031DD9032100312A402A20002100402AEF
:100480003C082000E70021008B1620006108FA3CA0
:10049000031D4D2AE2080319512AE10A0319E20A51
:1004A000532AE401E3012100BC0120008D1C5B2ADA
:1004B0002100BC0A20002100BD0120000D1D632A7F
:1004C0002100BD0A2000DA080319042B2100BC0812
:1004D00003196C2A2000042B2000DE01DD0121001D
:1004E000BD080319792A2000DB0A0319DC0A7E2AD9
:1004F000210020005B080319DC03DB0321003C081A
:100500002000DA00E008031D032B5F08313C031CC8
:10051000032BDF08031D8F2AE0080319032B21009A
:10052000C3013230C200200060082100C500200055
:100530005F082100C400F801F901F701FA0145083C
:10054000031DA52A44080319BF2A1030C600031052
:10055000C20DC30DF70DFA0D45087A02031DB22A2C
:1005600044087702031CBB2A4408F702031CFA0361
:100570004508FA020314F80DF90DC60BA72A7808EE
:10058000BE00043C0318C62A0430BE0020005C08EC
:100590002100C30020005B082100C200C5013E0805
:1005A000C400430845068039C700C31FDC2AC209BE
:1005B000C309C20A0319C30AC51FE32AC409C5092E
:1005C000C40A0319C50A1030C600F701FA01C30CAA
:1005D000C20C031CF12A4408F7070318FA0A45085D
:1005E000FA07FA0CF70CF90CF80CC60BE72AC71F30
:1005F000FE2AF809F909F80A0319F90A790820000E
:10060000DC007808DB00122B21003C082000DA0017
:100610005F082C3C031D0F2B600B0F2B122BDF0AE6
:100620000319E00ADC1B282BDC08031D1B2B5B08CD
:10063000003C0318282B5B085C040319272B5B087C
:100640000319DC03DB03D908031DD9031B2B362B4D
:10065000DC1F362B5B085C040319362BDB0A0319FD
:10066000DC0A59087F3C031DD90A2A2BE508031D23
:100670003C2BE6080319402B65080319E603E50344
:100680000B118031132821008C1022008C142100C2
:100690000C1022000C1021008C130C1322000C13E0
:1006A0008831200034282030850063308400000821
:1006B0000319672B0A30F800F701F70B5D2BF80BD5
:1006C0005C2B5F30F700F70B632B800B5A2B080075
:1006D00022008C102000EF080319722B22008C17C7
:1006E000742B200022008C130C140C108C170C148B
:1006F0000C100C140C100C140C100039F700210015
:1007000021080839FA0077087A0403198B2B220094
:100710008C178D2B210022008C130C140C10003927
:10072000F700210021080439FA0077087A04031938
:100730009D2B22008C179F2B210022008C130C1460
:100740000C100039F700210021080239FA0077085F
:100750007A040319AF2B22008C17B12B2100220041
:100760008C130C140C100039F700210021080139FA
:10077000FA0077087A040319C12B22008C17C32BC7
:10078000210022008C130C140C1021002008803949
:10079000F700FA0177087A040319D22B22008C178C
:1007A000D42B210022008C130C140C1021002008E3
:1007B0004039F700FA0177087A040319E32B220085
:1007C0008C17E52B210022008C130C140C10210037
:1007D00020082039F700FA0177087A040319F42B6E
:1007E00022008C17F62B210022008C130C140C1005
:1007F000210020081039F700FA0177087A0403195C
:10080000052C22008C17072C210022008C130C14BD
:100810000C10210020080839F700FA0177087A0443
:100820000319162C22008C17182C210022008C137F
:100830000C140C10210020080439F700FA01770885
:100840007A040319272C22008C17292C210022005E
:100850008C130C140C10210020080239F700FA0147
:1008600077087A040319382C22008C173A2C2100BF
:1008700022008C130C140C10210020080139F70001
:10088000FA0177087A040319492C22008C174B2CA3
:10089000210022008C130C140C108C140C131A3031
:1008A000F700F70B512C00000C171A30F700F70B6C
:1008B000572C000020000800EC0123009101951343
:1008C000151413084F3C0319682C2000EC0A230070
:1008D000013091009513151413084B3C0319732C28
:1008E0002000EC0A23000230910095131514130820
:1008F000493C03197E2C2000EC0A230003309100B0
:10090000951315141308523C0319892C2000EC0A86
:10091000230004309100951315141308413C03196A
:10092000942C2000EC0A2300053091009513151437
:1009300013084B3C03199F2C2000EC0A23000630BF
:100940009100951315141308553C0319AA2C200087
:10095000EC0A23002000ED010D19ED0AEE018D18BF
:10096000EE0A01302100B300200053232100A20130
:10097000A1012208033C031CEB2C031DC32C2108FE
:10098000833C031CEB2C2000EF010D19EF0A210022
:10099000A00120008D1CCF2C2100A00A20006F0890
:1009A0006D020319D62CEC0A6F08ED002100200817
:1009B00020006E020319E12CEC0A2100200820001F
:1009C000EE0001302100B300200053232100A10AD2
:1009D0000319A20AB92C20006C08F80088314628B7
:1009E000230091014F309300951315150B08F70064
:1009F0008B1355309600AA30960095149518FE2C4E
:100A0000151177088B04013091004B30930095133A
:100A100015150B08F7008B1355309600AA30960079
:100A200095149518112D151177088B04023091003B
:100A300049309300951315150B08F7008B135530AB
:100A40009600AA30960095149518242D1511770854
:100A50008B040330910052309300951315150B0849
:100A6000F7008B1355309600AA3096009514951810
:100A7000372D151177088B04043091004130930015
:100A8000951315150B08F7008B1355309600AA30F7
:100A90009600951495184A2D151177088B0405308A
:100AA00091004B309300951315150B08F7008B132D
:100AB00055309600AA309600951495185D2D1511A5
:100AC00077088B0406309100553093009513151567
:100AD0000B08F7008B1355309600AA30960095143A
:100AE0009518702D151177088B042000D901093055
:100AF0002300910020005908230093009513151539
:100B00000B08F7008B1355309600AA309600951409
:100B10009518882D151177088B042000ED01EC0144
:100B2000ED08031DC62D6C08013C031CC62D1030BA
:100B30006C072100A200003020006D3D2100A300C1
:100B4000053020006C07840020306D3D85000830A2
:100B500080002100A4002208230091002100240825
:100B600023009300951315150B08F7008B135530D0
:100B70009600AA30960095149518BC2D151177088B
:100B80008B042000EC0A0319ED0A902D2100A1012D
:100B9000A0012000ED01EC01ED08031D042E6C08FE
:100BA000013C031C042EEF01EE01EF08031D002E93
:100BB0006E080F3C031C002E203021002007A200ED
:100BC0000030213DA30022082300910055309300FE
:100BD000951315150B08F7008B1355309600AA30A6
:100BE000960095149518F22D151177088B042100A5
:100BF000A00A0319A10A2000EE0A0319EF0AD52D55
:100C0000EC0A0319ED0ACC2D88314C2822000D1670
:100C10002000EF016F08013C031CBD2E6F0B132E4B
:100C200022008D162000A4018B1BA4178B131A2100
:100C3000A41B8B1778082100A000A008031D232EF9
:100C40002000132E21002000EC016C080F3C031C37
:100C5000492E52306C07F8002030FA000318FA0AC7
:100C600078082100B2007A08B300273020006C0712
:100C70008400203085000318850A00082100B40094
:100C80003308850032088400340880002000EC0A14
:100C9000252E02302100B200FA30B3002000532389
:100CA0002100B20B4C2E3F30A005103020006F0702
:100CB0002100B200053020006F078400203085003D
:100CC0000318850A2100200880002008B30032089C
:100CD000230091002100200823009300951315158F
:100CE0000B08F7008B1355309600AA309600951428
:100CF0009518782E151177088B042000EC016C08EC
:100D00000F3C031CB02E6F0EF700F030F70577088C
:100D10006C07203E2100B200523020006C07840096
:100D2000203085000318850A00082100B30032082E
:100D3000230091002100330823009300951315151B
:100D40000B08F7008B1355309600AA3096009514C7
:100D50009518A82E151177088B042000EC0A7F2E19
:100D600002302100B200FA30B300200053232100EA
:100D7000B20BB32E2000EF0A0A2E22000D128D12A4
:100D8000883120004F280930230091009513151455
:100D900013082000D9002100A101A0012000ED01CD
:100DA000EC01ED08031D312F6C08013C031C312FB1
:100DB00005306C07840020306D3D850010306C07D5
:100DC0002100A400003020006D3D2100A500240872
:100DD0002300910095131514130880002000EF01E3
:100DE000EE01EF08031D2D2F6E080F3C031C2D2F65
:100DF0006C0D2100A20020006D0D2100A300A20DAA
:100E0000A30DA20DA30DA20DA30DF030A20520008D
:100E10006E0821002207F80020006F082100233D02
:100E2000FA007808073E840020307A3D85002030A3
:100E30002007A4000030213DA500240823009100D4
:100E400095131514130880002100A00A0319A10AA4
:100E50002000EE0A0319EF0AF12EEC0A0319ED0A3D
:100E6000D12E2100A101A0012000ED01EC01ED082F
:100E7000031D522F6C08013C031C522F05306C07D8
:100E8000840020306D3D850000087F39103C031838
:100E90004E2F2100A00A0319A10A2000EC0A031911
:100EA000ED0A372F21002008F80088312000522851
:100EB000EE016C08ED00ED0DEE0DED0DEE0DED0DFE
:100EC000EE0DED0DEE0DED0DEE0DE030ED056C08C7
:100ED0007F3C031D6F2F0F30EE00FF30ED00EF0160
:100EE0006E082100A10020006D082100A000200054
:100EF00068230800E508031DA52FE608031DA52F9C
:100F00001330E6008830E50059082300910095135E
:100F100015141308200059020319A52F09302300C6
:100F200091002000590823009300951315150B0814
:100F3000F7008B1355309600AA309600951495183B
:0E0F40009F2F151177088B0420008831A928F7
:10100000850184011F308305F43021009900200000
:10101000D901DA01DC01DB01DE01DD01E001DF01E4
:10102000E201E101E401E3011330E6008830E5006C
:1010300023008C018D012200920191019401930102
:101040002000E701F03021009900FF3024008D00DE
:10105000210095130D1222000D1221008D12220085
:101060008D1280312000432B883164302100B30081
:101070008031200053238831EF012100A101A0011C
:10108000803120006823883180315C2C8831F80859
:10109000031950288031F02C88318031062E883198
:1010A0008031C32E88315908EC00803158278831AF
:1010B00021001508C039043895000730200095003C
:1010C0008B16C0308B04E801680859020319A72861
:1010D0005908680203188A286808590203198928E0
:1010E000E80A6808EC008031582788315808033C2A
:1010F000031D822805302100B300803120005323D6
:101100008831892808302100B30080312000532322
:101110008831A728680859020319A728E803680836
:10112000EC008031582788315808033C031DA02863
:1011300005302100B3008031200053238831A728D7
:1011400008302100B30080312000532388318031E2
:081150007A2F88316428630046
:020000040001F9
:04000E000439FF1E94
:00000001FF
